:1000000000308A00492A0000831A0A28A500030E3E
:10001000A6000F288312A500030EA600A6140A0846
:10002000AD008A018313A50E0408A7002008A800CC
:100030002108A9002208AA002308AB002408AC006C
:1000400083128C308400801C27288C183C282708B9
:1000500084002808A0002908A1002A08A2002B0873
:10006000A3002C08A4002D088A00260E830083120A
:10007000250EA61883160900B30A6D08643C3302E6
:1000800003194928031C49288316871183128715F1
:100090004D2883168711831287116E08643C330242
:1000A00003195928031C59288316071083120714B3
:1000B0005D2883160710831207106F08643C330213
:1000C00003196928031C6928831687108312871473
:1000D0006D2883168710831287103308643C031D34
:1000E0007228B3010130F3008C108A112728A10176
:1000F000A201A001A3017A08031D81287908031930
:100100009B281030FB000310F70DF80DA00DA30D78
:100110007A082302031D8E2879082002031C9728E1
:100120007908A002031CA3037A08A3020314A10DFB
:10013000A20DFB0B832800343208F7003108F600CB
:100140003008F5002F08F4004130FB00C630FA00FB
:100150004E30F9006D30F80020308316A400A00165
:10016000A101A201A30177088312A3007608A200CF
:100170007508A1007408A0000310201CCF2878087F
:100180008316A00779080318790FA1077A080318C6
:100190007A0FA2077B0803187B0FA307831283162D
:1001A000A30CA20CA10CA00C8312A30CA20CA10CFA
:1001B000A00C8316A40BDD28DF288312BC28831231
:1001C00039302007AF002108B0003030031831303B
:1001D000B0072208B100003003180130B10723082E
:1001E000B200003003180130B2073108A000320815
:1001F000A100A201A3013208F6003108F50032087F
:10020000F8003108F7007F30FA00FF30F90077205E
:100210002008A1002308A20000341030FD00A00136
:10022000A301FA0CF90C031C1B297B08A007031877
:10023000A30A7C08A307A30CA00CA20CA10CFD0B25
:1002400011290034A001A101A201A3018316A40178
:10025000A501A601A70123082204210420040319F3
:1002600063292030A8000310F90DFA0DFB0DFC0DD9
:10027000A40DA50DA60DA70D23082702031D4A29CD
:1002800022082602031D4A2921082502031D4A29A6
:1002900020082402031C5B292008A4022108031C57
:1002A000210FA5022208031C220FA6022308031C0B
:1002B000230FA70203148312A00DA10DA20DA30DFD
:1002C0008316A80B3329A430840083120034013034
:1002D000D4070318D50A0319D60A0319D70A6008E8
:1002E0005402031DA22961085502031DA2296208B8
:1002F0005602031DA22963085702031DA229D70134
:10030000D601D501D401720803198A29013A0319CB
:100310009629A129E90AE91B95296C086902031CA1
:1003200095296C08E9000130F200A229E903E91BD4
:100330009D2969086602031CA0296608E900F201EC
:10034000A229A2299C202208F5002108F4002208F5
:10035000F8002108F700FA010A30F9007720200898
:10036000EF00CA2B0130CC070318CD0A0319CE0ABF
:100370000319CF0A58084C02031DED2959084D02F4
:10038000031DED295A084E02031DED295B084F029B
:10039000031DED29CF01CE01CD01CC017008031959
:1003A000D529013A0319E129EC29E70AE71BE029DD
:1003B0006A086702031CE0296A08E7000130F000C0
:1003C000ED29E703E71BE82967086402031CEB2912
:1003D0006408E700F001ED29ED299C202208F500D2
:1003E0002108F4002208F8002108F700FA015B3028
:1003F000F90077200A302007ED00CB2B0130D00721
:100400000318D10A0319D20A0319D30A5C0850024F
:10041000031D392A5D085102031D392A5E08520264
:10042000031D392A5F085302031D392AD301D20163
:10043000D101D00171080319212A013A03192D2A8B
:10044000382AE80AE81B2C2A6B086802031C2C2AAD
:100450006B08E8000130F100392AE803E81B342A70
:1004600068086502031C372A6508E800F101392A8B
:10047000392A9C202208F5002108F4002208F800FF
:100480002108F700FA013C30F90077202008EE003F
:10049000CC2B84011F3083051F130030831691007D
:1004A00083129A0107309900AE010130AF00B0010C
:1004B000B101B201B301CC01CD01CE01CF01D00118
:1004C000D101D201D301D401D501D601D7010A301F
:1004D000E4001430E5001E30E600E701E801E90120
:1004E0005030EA003230EB006430EC00F001F101F2
:1004F000F2011F1300308316910083121F10181091
:100500008316871683129501960183160108C03958
:100510008100831290014830A100043892006430B9
:100520008316920007118312071183168C14C030B2
:1005300083128B04C301C201C101C001C701C601FE
:10054000C501C401CB01CA01C901C801B701B60187
:100550000330B500E830B400BB01BA010330B90084
:10056000E830B800BF01BE010330BD00E830BC0078
:10057000C008031D412BC108031D412BC208031DE8
:10058000412BC308031D412B9C202208F5002108A4
:10059000F4002208F8002108F700FA010A30F900F7
:1005A00077202008F5002308F60001302007F70027
:1005B0002308F8000318F80A7808FA007708F90009
:1005C0002730FC001030FB000D21C301C2012208BE
:1005D000C1002108C0009C202208F5002108F40079
:1005E0002208F8002108F700FA01C830F900772046
:1005F0002008F5002308F60001302007F700230843
:10060000F8000318F80A7808FA007708F9000130B2
:10061000FC00F430FB000D21B701B6012208B50043
:100620002108B4006430EA000A30E4000310370CFB
:10063000F700360CF600350CF500340CF4006408B5
:100640006A02F8007708FC007608FB007508FA00DB
:100650007408F9008316A301A201A1017808A00083
:10066000831222212308DB002208DA002108D900A6
:100670002008D8006408E700CF01CE01CD01CC01ED
:10068000F001C408031DC62BC508031DC62BC608F0
:10069000031DC62BC708031DC62B9C202208F5008E
:1006A0002108F4002208F8002108F700FA0164305C
:1006B000F90077202008F5002308F6000130200714
:1006C000F7002308F8000318F80A7808FA007708FA
:1006D000F9000330FC00E830FB000D21C701C60122
:1006E0002208C5002108C4009C202208F50021082A
:1006F000F4002208F8002108F700FA01C830F900D8
:1007000077202008F5002308F60001302007F700C5
:100710002308F8000318F80A7808FA007708F900A7
:10072000FC01FA30FB000D21BB01BA012208B9001F
:100730002108B8006430EB00E50103103B0CF70022
:100740003A0CF600390CF500380CF40065086B0221
:10075000F8007708FC007608FB007508FA007408BA
:10076000F9008316A301A201A1017808A000831259
:1007700022212308DF002208DE002108DD002008F6
:10078000DC00D301D201D101D001F101F30803193A
:10079000E52B6729B229FE29F301FF30C007031CAE
:1007A000C107031CC207031CC307FF30C407031C97
:1007B000C507031CC607031CC707FF30C807031C77
:0E07C000C907031CCA07031CCB07B82A630035
:02400E00E73F8A
:00000001FF
